:020000040000FA
:10040000BFFFDFFFFFFFFFFFFFFFFFFFFFFFFFFF5C
:10041000FFFFFFFFFFFFFFFFFFFFFFFFFFFFFFFFEC
:10042000FFFFFFFFFFFFFFFFFFFFFFFFFFFFFFFFDC
:10043000FFFFFFFFFFFFFFFFFFFFFFFFFFFFFFFFCC
:10044000FFFFFFFFFFFFFFFFFFFFFFFFFFFFFFFFBC
:10045000FFFFFFFFFFFFFFFFFFFFFFFFFFFFFFFFAC
:020000040000FA
:10800000500A0020258300002D8300002F830000EC
:10801000318300003383000035830000000000003E
:108020000000000000000000000000006582000069
:108030003983000000000000C1820000D1960000DA
:10804000ED8B0000FD8B00000D8C00001D8C0000EE
:108050002D8C00003D8C00004D8C00005D8C0000DC
:108060006D8C00007D8C00008D8C00009D8C0000CC
:10807000AD8C0000BD8C0000CD8C0000DD8C0000BC
:1080800075880000898800003F8300003F8300005E
:108090003F8300003F8300003F8300003F830000D8
:1080A000BD880000D3880000E9880000FF88000038
:1080B000158900003F890000558900003F830000BA
:1080C0003F8300003F8300003F8300003F830000A8
:1080D0003F8300003F8300003F8300003F83000098
:1080E0003F8300003F8300003F8300003F83000088
:1080F0003F8300003F8300003F8300003F83000078
:108100003F8300003F8300003F8300003F83000067
:108110003F8300003F8300003F8300003F83000057
:108120003F8300003F8300003F8300003F83000047
:108130003F8300003F8300003F8300003F83000037
:108140003F8300003F8300003F8300003F83000027
:108150003F8300003F8300003F8300003F83000017
:108160003F8300003F8300003F8300003F83000007
:108170003F8300003F8300003F8300003F830000F7
:108180003F8300003F8300003F8300003F830000E7
:108190003F8300003F8300003F8300003F830000D7
:1081A0003F8300003F8300003F8300003F830000C7
:1081B0003F8300003F8300003F8300003F830000B7
:1081C0003F8300003F8300003F8300003F830000A7
:1081D0003F8300003F8300003F8300003F83000097
:1081E0003F8300003F8300003F8300003F83000087
:1081F0003F8300003F8300003F8300003F83000077
:108200003F8300003F8300003F8300003F83000066
:108210003F8300003F830000058E00003F83000085
:10822000D58F00003F8300003F8300003F830000A4
:108230003F8300003F8300003F8300003F83000036
:108240003F8300003F8300003F8300003F83000026
:10825000DFF80CD000F0ECF8004800477DA10000EA
:10826000500A00202C4B19680868B0E8F04F80F3E2
:108270000988BFF36F8F4FF0000080F311887047BB
:108280000000000008480068006880F308884FF08C
:10829000000080F3148862B661B6BFF34F8FBFF35E
:1082A0006F8F00DF00BF00BF08ED00E0DFF80C00BB
:1082B000016841F470010160704700BF88ED00E083
:1082C000EFF30980BFF36F8F134B1A681EF0100F86
:1082D00008BF20ED108A20E9F04F106009B44FF07C
:1082E000500080F31188BFF34F8FBFF36F8F03F0FF
:1082F00065FB4FF0000080F3118809BC196808681D
:10830000B0E8F04F1EF0100F08BFB0EC108A80F3F9
:108310000988BFF36F8F70471881FF1FEFF3058047
:10832000704700000648804706480047FEE7FEE722
:10833000FEE7FEE7FEE7FEE7FEE7FEE7FEE7FEE715
:10834000D1970000518200002DE9F05F0546002022
:1083500092469B4688460646814640241BE02846B6
:1083600041464746224600F053F853465A46C01A43
:10837000914110D311461846224600F016F82D1AE6
:1083800067EB01084F4622460120002100F00DF85E
:1083900017EB00094E41201EA4F10104DFDC484622
:1083A00031462A464346BDE8F09F202A04DB203AA6
:1083B00000FA02F1002070479140C2F1200320FA38
:1083C00003F319439040704740EA01039B0703D031
:1083D00009E008C9121F08C0042AFAD203E011F804
:1083E000013B00F8013B521EF9D27047D2B201E0C6
:1083F00000F8012B491EFBD270470022F6E710B5AA
:1084000013460A4604461946FFF7F0FF204610BD02
:10841000202A04DB203A21FA02F00021704721FAD9
:1084200002F3D040C2F12002914008431946704740
:10843000064C074D06E0E06840F0010394E80700B1
:1084400098471034AC42F6D3FFF706FF64C600002D
:1084500084C6000030B58C1810F8012B12F00F0301
:1084600001D110F8013B120906D110F8012B03E0ED
:1084700010F8015B01F8015B5B1EF9D101E001F826
:10848000013B521EFBD1A142E6D3002030BD026861
:1084900061F308020260704708B50021009102E014
:1084A0000099491C009100998142F9D308BD000050
:1084B000014604480078084008B1012070470020B8
:1084C000FCE700003C40054070B50446002564B957
:1084D0001648007800F00700052801D1AD1F22E002
:1084E00001201249091D08701DE01048DA300068AB
:1084F000C0F3C01030B94FF48051082000F073F879
:10850000054605E04FF48051012000F06CF8054667
:108510004DB900200549091D08704FF480512020F5
:1085200000F061F80546284670BD00002640054071
:1085300070B5044614B96FF0020514E02079C10942
:108540000A48006861F3C71008490860606808605D
:10855000207820B90120FFF7B7FF054603E000208F
:10856000FFF7B2FF0546284670BD000000410540F8
:108570000146002009B9C01E22E000224A604A6874
:1085800022F080024A604A6822F003024A60132304
:108590004A6863F310224A604A6822F0704202F18E
:1085A00080524A604A6822F0706202F180724A602A
:1085B0004A6822F4700202F580124A6001220A70B1
:1085C000704770B504460D462946204600F0B4FFBA
:1085D00001F098F870BD10B50446204601F016F879
:1085E00001F090F810BD18B503460A46002000902F
:1085F0006FF0070409E01846FFF75AFF012801D180
:10860000002405E00098401C009000989042F2D9A8
:1086100000BF204618BD000070B504460025F4B91F
:108620001548007800F00700032801D1AD1F20E0B5
:108630001148DA300068C0F3C01058B90E48001D68
:10864000007810B96FF0050513E001200A490C31DC
:1086500008700EE0012008490C31087009E0002084
:1086600005490C3108704FF480510820FFF7BBFF1B
:108670000546284670BD00002640054070B50446FA
:1086800014B96FF0020514E0E0780B4908706078C7
:1086900040F08000A178084308490870207820B98C
:1086A0000120FFF7B9FF054603E00020FFF7B4FF04
:1086B0000546284670BD0000A240054050CC04404D
:1086C0000146002009B9C01E06E001220A700022FE
:1086D0008A704A700522CA7070470346012A05D184
:1086E0000120884000F03F00D86104E0012088406C
:1086F00000F03F0058630020704782690A4382619E
:10870000704701607047F0B5034600200AB9C01EEB
:1087100028E003F1400505EB811556682E6003F152
:10872000440505EB811596682E60968A156945EA21
:10873000064603F1480505EB81152E6003F15C0543
:1087400005EB8114D6681568354396693543D669BB
:10875000354341F20F363540266841F20F37BE43AC
:1087600035432560F0BD000010B5104A00211048C7
:1087700000F02AF84FF4807200210D4800F02CF828
:108780000C4A01210A4800F017F84FF480720121C9
:10879000074800F021F8012200210548FFF79DFF5E
:1087A000012211460248FFF798FF10BD1480FF1FF9
:1087B00000300540A881FF1F034603F1440000EB91
:1087C0008110026000207047034603F1400000EB77
:1087D000811002600020704710B5034603F1480085
:1087E00000EB8114206862F31F402060002010BD60
:1087F0000146002009B9C01E0AE000220A604A6052
:108800008A60CA6001220A6100224A618A61CA61E3
:108810007047000010B502210148FFF76EFF10BD40
:1088200000300540014600220F48006861F3030054
:108830000D4B186010E0521C0C48006AC0F3026334
:108840000B480068D84044F62063B0FBF3F0904238
:1088500002D26FF0070070470348006800F00F0075
:108860008842E8D10020F6E71804014000400540A6
:1088700044FEFF1F10B5012000F080F8012801D14F
:1088800000F074F810BD000010B5022000F076F87A
:10889000012805D103A001F00FF8022000F066F8CE
:1088A00010BD0000455854494E545F4348303120B4
:1088B000696E74657272757075740A0010B54FF444
:1088C000807000F05BF8012802D1000200F04EF841
:1088D00010BD10B54FF4007000F050F8012802D11F
:1088E000400200F043F810BD10B54FF4806000F076
:1088F00045F8012802D1800200F038F810BD10B50B
:108900004FF4006000F03AF8012802D1C00200F0F4
:108910002DF810BD10B54FF4805000F02FF801284D
:108920000CD10103042000F0CFF84FF48051022055
:1089300000F0CAF84FF4805000F018F810BD10B5E0
:108940004FF4005000F01AF8012802D1400300F063
:108950000DF810BD10B54FF4804000F00FF801285D
:1089600002D1800300F002F810BD00000249896DB9
:108970000143014A916570470010054001460448D3
:10898000406D084008B1012070470020FCE700005E
:1089900000100540012905D1054A12688243044BA5
:1089A0001A6004E0024A12680243014B1A607047E1
:1089B00000800440012905D1054A52688243044BD6
:1089C0005A6004E0024A52680243014B5A60704701
:1089D0000080044030B503460C46002115E0012517
:1089E0008D4025407DB10A4D05EB831505EB8100D7
:1089F000012A04D1058845F40045058003E0058877
:108A0000C5F30E0505804D1CE9B21029E7D330BD32
:108A1000003C05402DE9F04104460F4600200AB90C
:108A2000C01E4CE0002148E04FF0010C0CFA01FCA4
:108A30000CEA070CBCF1000F3BD0B2F800C0B2F852
:108A400002804CEA080CB2F804804CEA080CB2F838
:108A500006804CEA080CB2F80A804CEA080CB2F81E
:108A60000E804CEA080CB2F810804CEA080CB2F800
:108A700008804CEA080545F27723B2F814C04CEAA6
:108A8000050543F40043B2F812C04CEA050543F46F
:108A90008063DFF830C00CEB841C0CEB8106B6F869
:108AA00000C02CEA030C05EA03084CEA080CA6F8FF
:108AB00000C001F1010C0CF0FF011029B4D3BDE896
:108AC000F0810000003C05400246054B03EB02101C
:108AD000B0F80008084008B1012070470020FCE70A
:108AE0000030054010B5044B102404FB00321388FD
:108AF0000B43138010BD00000A38054030B5034613
:108B000000200BE0012585400D402DB1054D05EB02
:108B1000831505EB80042280451CE8B21028F1D3B0
:108B200030BD0000023C054010B5044B102404FB8E
:108B3000003213880B43138010BD00000838054035
:108B40000549098848F6FF72114000F4E0421143DC
:108B5000014A118070470000F83B054001460020A3
:108B600009B9C01E0BE000220A804A80CA808A82AE
:108B70008A810A814A81CA810A828A804A82704730
:108B800030B50146002009B9C01E2AE0B1F9023013
:108B90000F2B02DD6FF0020023E04B88114C0425FF
:108BA00015FB03421368C3F3080340F2FF14A3420A
:108BB00008D10B881360B1F902400B4D4B6845F8A2
:108BC00024300EE00B881468C4F30804A34206D1D5
:108BD000B1F90240044D4B6845F8243001E06FF0D4
:108BE000010030BD5C100540A882FF1F10B502498E
:108BF0000868804710BD0000A882FF1F10B5024919
:108C00004868804710BD0000A882FF1F10B50249C8
:108C10008868804710BD0000A882FF1F10B5024978
:108C2000C868804710BD0000A882FF1F10B5024928
:108C30000869804710BD0000A882FF1F10B50249D7
:108C40004869804710BD0000A882FF1F10B5024987
:108C50008869804710BD0000A882FF1F10B5024937
:108C6000C869804710BD0000A882FF1F10B50249E7
:108C7000086A804710BD0000A882FF1F10B5024996
:108C8000486A804710BD0000A882FF1F10B5024946
:108C9000886A804710BD0000A882FF1F10B50249F6
:108CA000C86A804710BD0000A882FF1F10B50249A6
:108CB000086B804710BD0000A882FF1F10B5024955
:108CC000486B804710BD0000A882FF1F10B5024905
:108CD000886B804710BD0000A882FF1F10B50249B5
:108CE000C86B804710BD0000A882FF1F10B5044666
:108CF00004F0010048B100BF40F223101A49086097
:108D000043F21020086000BF00BF04F0020028B149
:108D100000BF16481649086100BF00BF04F00400F8
:108D200030B100BF4AF201501249088000BF00BFB5
:108D300004F0100018B14AF2085000F04FFB04F0A4
:108D4000400018B14AF2035000F048FB04F08000E4
:108D500040B100BF77200849086007490831086022
:108D600000BF00BF10BD0000000401400100A5A528
:108D700000800440FC3B05400408054010B5044653
:108D800004F0010028B100BF00201949086000BFAD
:108D900000BF04F0020028B100BF16481649086160
:108DA00000BF00BF04F0040030B100BF4FF4254005
:108DB0001249088000BF00BF04F0100018B14AF249
:108DC000085000F0FDFA04F0400018B14AF20350D8
:108DD00000F0F6FA04F0800040B100BF76200849A8
:108DE000086007490831086000BF00BF10BD0000DF
:108DF000000401400000A5A500800440FC3B0540A4
:108E00000408054030B59FB0002501215D4800F001
:108E1000CFFA012845D101215A4800F0A7F95AA0FC
:108E200000F04AFD04AA4021564800F0C1F900288C
:108E300037D1002405E00EA8015D5AA000F03CFDEA
:108E4000641C082CF7DB0598C0B28DF8000004986C
:108E5000019008208DF80100DDE90E01CDE9020145
:108E60000498B0F5F66F07D100234F4A04A94F4884
:108E7000006802F03FFF06E002234B4A69464C4877
:108E8000006802F037FF00BF4748006838B14FF074
:108E9000805048490860BFF34F8FBFF36F8F00BF0A
:108EA00000BF0421374800F083FA012803D10421D0
:108EB000344800F05BF91021324800F079FA0128BB
:108EC00045D110212F4800F051F93BA000F0F4FCEF
:108ED00004AA41212B4800F06BF9002837D1002467
:108EE00005E00EA8015D2FA000F0E6FC641C082C34
:108EF000F7DB0598C0B28DF80000049801900820B7
:108F00008DF80100DDE90E01CDE902010498B0F50C
:108F1000F66F07D10223244A04A92448006802F00E
:108F2000E9FE06E00223204A69462148006802F073
:108F3000E1FE00BF1C48006838B14FF080501D4969
:108F40000860BFF34F8FBFF36F8F00BF00BF40219A
:108F50000C4800F02DFA012807D14021094800F003
:108F600005F92946074800F003F94FF400210548A8
:108F700000F01EFA012803D1C104024800F0F6F8FF
:108F80001FB030BD009002405278204649464F5FE6
:108F900030206E6577206D6573736167652D3E0DBA
:108FA0000A000000257820000C80FF1F0080FF1FB2
:108FB0000480FF1F04ED00E05278204649464F5FD1
:108FC00031206E6577206D6573736167652D3E0D89
:108FD0000A00000030B59FB000250121504800F084
:108FE000E7F9012838D101214D4800F0BFF84DA024
:108FF00000F062FC04AA4021494800F0D9F858BBAF
:10900000002405E00EA8015D4DA000F055FC641C95
:10901000082CF7DB0598C0B28DF800000498019089
:1090200008208DF80100DDE90E01CDE902010223DF
:10903000444A69464448006802F05CFE00BF41486B
:10904000006838B14FF0805040490860BFF34F8F3F
:10905000BFF36F8F00BF00BF0421314800F0A8F9B3
:10906000012803D104212E4800F080F810212C485B
:1090700000F09EF9012838D11021294800F076F837
:1090800033A000F019FC04AA4121254800F090F813
:1090900058BB002405E00EA8015D29A000F00CFCDF
:1090A000641C082CF7DB0598C0B28DF8000004980A
:1090B000019008208DF80100DDE90E01CDE90201E3
:1090C0000223204A69462048006802F013FE00BFD0
:1090D0001C48006838B14FF080501C490860BFF34D
:1090E0004F8FBFF36F8F00BF00BF40210C4800F0CF
:1090F0005FF9012807D14021094800F037F82946D7
:10910000074800F035F84FF40021054800F050F909
:10911000012803D1C104024800F028F81FB030BD77
:10912000009402405278204649464F5F30206E65D9
:1091300077206D6573736167652D3E0D0A00000031
:10914000257820001080FF1F0880FF1F04ED00E03D
:109150005278204649464F5F31206E6577206D6515
:1091600073736167652D3E0D0A000000016570474D
:10917000C0F8D010704700000146AC31486C4FF683
:10918000FC731840084BC21808684FF6FC7318406F
:10919000054B1844121A0869AC39C0F30220034B7E
:1091A000185CB2FBF0F0704700B002405CC60000F3
:1091B0002DE9FC5F04460F4615464FF000080020DD
:1091C000009083466FF00209002D7CD08146402F2D
:1091D0002ED1D4F8A00000F4FE0008B96FF0020907
:1091E000B9F1000F06D1D4F8A40000F07F0008B94F
:1091F0006FF00809B9F1000F6CD1A0346068C0F3BA
:10920000052B20684FF6FC710840664900EB010809
:10921000E06900F007006449085C1BFB0088E06916
:10922000A03C00F0070008306049085C009051E065
:10923000412F2ED1D4F8B00000F4FE0008B96FF031
:109240000209B9F1000F06D1D4F8B40000F07F0094
:1092500008B96FF00809B9F1000F3BD1B03460686C
:10926000C0F3052B20684FF6FC7108404D4900EB18
:109270000108E068C0F302104B49085C1BFB008842
:10928000E068B03CC0F3021008304849085C009028
:1092900020E02046FFF770FFB84202D86FF00209C5
:1092A00018E054F8AC0F4FF6FC7108403D4900EB54
:1092B00001082069C0F302203B49085C07FB0088D5
:1092C0002069AC3C00E057E0C0F302200830374989
:1092D000085C0090B9F1000F61D146463068C0F3D8
:1092E00080706860686820B93068C0F38A40286080
:1092F00003E0306820F0604028603068C0F34070C0
:10930000A8603068C00F286108F10406308880B278
:10931000E8613068C0F30340E8602449E868085C0D
:10932000A866A96E0098814201D90098A8663068A5
:10933000C0F3005068613068C0F34050A8613068E5
:10934000C0F3066028623068C00F686208F1080642
:1093500001964FF0000A08E0019810F80A1005F194
:10936000280000F80A100AF1010AA86E5045F3D847
:10937000402F02D1C4F8A8B011E0412F02D1C4F8A7
:10938000B8B00CE0202F04D20120B840C4F89800F7
:1093900005E007F01F0101208840C4F89C00484602
:1093A000BDE8FC9F00B002405CC600004CC6000057
:1093B00002460020136D0B4003B1012070470000EE
:1093C00004490988814341F42541034AA2F8FE1368
:1093D00070470000FE4305400040054003490988EE
:1093E0000143034AA2F8FE1370470000FE43054004
:1093F0000040054000B587B00020ADF8060001AA86
:109400004FF480610220FFF705FB07B000BD00B5F7
:1094100087B00220ADF806000420ADF8080001AACC
:1094200001020220FFF7F6FA07B000BD00BF704747
:1094300030B502466FF00200A9B38B68082B03D148
:10944000CB68B3F5805F2ED00B68012B06D18B68FB
:1094500023B94B693BB34B69022B24D0D1E90034CB
:1094600023438C6823434C6A2343CC6823430C6911
:10947000234353600C8B04F470448B6A23434FF2F4
:1094800003042340D4684FF20305AC432343D36065
:109490000C6A4B692343CC6923430C7E04F00C0413
:1094A00023439361002030BD01466FF0020099B163
:1094B00000220A604A6008228A600022CA600A61AB
:1094C0004A614FF440528A614FF48062CA610022BF
:1094D0000A624A628A6200207047000010B500F0FC
:1094E000010353B1134B1B6862F30203114C236059
:1094F00023461B6861F30613236000F0020353B197
:109500000C4B1B6862F312430A4C236023461B6812
:1095100061F31653236000F0040353B1054B1B683D
:1095200062F31A63034C236023461B6861F31E73C6
:10953000236010BD000805402DE9FF4104460D469B
:1095400000262E48006803902C48406802902B4863
:10955000806801902948C06800902948007800F090
:109560000700052816D10126264824490860C012A4
:1095700048608860C86022482638006AC0F30261EB
:1095800021480068C8404CF25031B0FBF1F7384632
:10959000FEF782FF1A482638006AA04305EA040154
:1095A00008431749263908620846006AC0F3026179
:1095B00015480068C8404CF25031B0FBF1F738460E
:1095C000FEF76AFF012E17D10C4903980860029834
:1095D0004860019888600098C86009482638006A89
:1095E000C0F3026108480068C8404CF25031B0FB3B
:1095F000F1F73846FEF750FFBDE8FF8100800440D8
:10960000264005400EFAFFFF44FEFF1F7FB50446CB
:1096100000252B480068039029484068029028489C
:10962000806801902648C06800902648007800F0C5
:109630000700052801D0052C16D101252248204914
:109640000860C01248608860C8601E482638006AFA
:10965000C0F302611D480068C8404CF25031B0FBB5
:10966000F1F63046FEF718FF164804701548263804
:10967000006AC0F3026115480068C8404CF25031DE
:10968000B0FBF1F63046FEF707FF012D17D10C496C
:109690000398086002984860019888600098C86044
:1096A00008482638006AC0F3026108480068C840CC
:1096B0004CF25031B0FBF1F63046FEF7EDFE7FBDC7
:1096C00000800440264005400EFAFFFF44FEFF1FC5
:1096D00010B500BF502080F31188BFF34F8FBFF348
:1096E0006F8F00BF02F0E4FC18B14FF080500449C6
:1096F000086000BF002080F3118800BF10BD00008B
:1097000004ED00E070B52B4D2D6805F001051DB18D
:10971000294D2A4E356002E0294D284E3560294DED
:109720002D7805F00700062840D2DFE800F0030896
:109730000C11151A214D2D68234E356037E0234D4D
:10974000214E356033E04FF400451F4E35602EE06A
:10975000194D1D4E35602AE04FF400451A4E356014
:1097600025E0184DDA352D68C5F30722154D263D45
:10977000D5F800512B0F134DDA352D6805F0030491
:10978000104D263DD5F8005105F080050DB90A4968
:1097900001E00A4D2968651CB1FBF5F5561C7543BF
:1097A0005E1CB5FBF6F5084E356000E000BF00BF5B
:1097B00070BD0000840601400024F40048FEFF1F35
:1097C000002D31012640054044FEFF1F00127A00A3
:1097D00000B50748006840F4700005490860FFF7CD
:1097E00091FF4FF4004002498039086000BD00003D
:1097F00088ED00E002461068084008B1012070477B
:109800000020FCE72DE9F04781460D4617469A46B1
:109810006FF0020875B36FB3D9F80C0000F48056EE
:1098200016B1B6F5805F25D1002416E0534601221B
:109830008021484600F021F88046B8F1000F00D0A2
:109840000DE026B9295D484600F033F804E035F80C
:109850001410484600F02DF8641CBC42E6D300BF4B
:10986000B8F1000F06D1534601224021484600F0CE
:1098700004F880464046BDE8F087F8B505460E4638
:1098800014460027002000900AE00098984204D96E
:10989000581C10B16FF0070708E00098401C0090BA
:1098A00031462846FFF7A6FFA042EED100BF38465A
:1098B000F8BD021D118070470FB4054B10B503A908
:1098C000044A029800F04CF810BC5DF814FB00004C
:1098D000999F0000A481FF1F002807DB00F01F02F2
:1098E00001219140024A430942F8231070470000C9
:1098F00080E200E000280DDB00BF00BF00F01F0287
:10990000012191404209920002F1E022C2F80011C7
:1099100000BF00BF7047000010B5002804DB0A0735
:10992000130E054A135406E00A07140E034A00F00A
:109930000F031B1FD45410BD00E400E018ED00E03D
:1099400002E008C8121F08C1002AFAD17047704708
:10995000002001E001C1121F002AFBD17047000066
:109960002DE9FF4F8DB00F460546002606E025285D
:109970000BD0DDE90F1290476D1C761C287800286B
:10998000F5D111B03046BDE8F08F0024A246A146C3
:109990000122EC4900E0044315F8013F203B02FAA4
:1099A00003F00842F7D128782A2810D06FF02F0250
:1099B0002878A0F13001092914D80AEB8A0102EBBA
:1099C000410144F0020400EB010A6D1CF0E701CFF5
:1099D0005FEA000A03D544F40054CAF1000A44F0D7
:1099E00002046D1C28782E2817D115F8010F44F0B9
:1099F00004042A280ED06FF02F022878A0F130013D
:109A000009290AD809EB890102EB410100EB0109A0
:109A10006D1CF2E757F8049B6D1C28786C280FD05A
:109A200006DC4C2817D068280DD06A2814D104E031
:109A3000742810D07A280FD10DE044F400140AE005
:109A400044F4801401E044F440146978814202D166
:109A500004F580146D1C6D1C2A786E2A1FD00CDC56
:109A6000632A31D004DC002A8BD0582A11D1A3E01C
:109A7000642A68D0692A0CD165E0732A2ED004DCF0
:109A80006F2A73D0702A04D19BE0752A6FD0782A90
:109A90006ED01046DDE90F129047761C50E1C4F3FA
:109AA0000250022806D0032809D0042801CF09D08B
:109AB000066045E101CFF117C0E9006140E101CF47
:109AC00006803DE106703BE117F8040B8DF80000BD
:109AD00000208DF80100EB46012003E057F804BB9D
:109AE0004FF0FF3061074FF0000102D40DE008F1A4
:109AF0000101884649450FDA8045F8DB1BF808105C
:109B00000029F4D108E008F1010188468142FADB1E
:109B10001BF808100029F6D1DDE90F23AAEB080095
:109B20008146214600F036F9304400EB080604E097
:109B3000DDE90F121BF8010B9047B8F10108F7D2CD
:109B400021464846F7E00A21C4F302534FF0000BC8
:109B50000891022B04D001CFC117032B09D00AE0D2
:109B6000FF1D27F00707F7E8020108E032E01FE0D9
:109B700020E000B2C117042B01D140B2C117031E6F
:109B800071F1000307DA4FF0000CD0EB0C006CEB26
:109B900001012D2302E0230504D52B238DF8243069
:109BA000012303E0E30701D02023F7E7984658E0BC
:109BB0000A2110E010210EE010204FF0000B089059
:109BC0000CE010214FF0000B44F004044FF00809A2
:109BD000089103E008214FF0000B0891C4F30253F1
:109BE000022B04D001CF0021032B06D006E0FF1D7D
:109BF00027F00707F7E8020103E080B2042B00D149
:109C0000C0B24FF0000823072BD5702A07D0DDF82B
:109C100020C08CF0100C5CEA0B0C05D00EE0402349
:109C20008DF82430012308E050EA010306D03023E8
:109C30008DF824308DF8252002239846DDF820C0C9
:109C40008CF0080C5CEA0B0C0BD150EA010301D13B
:109C5000630706D530238DF824304FF00108A9F1B1
:109C60000109582A04D038A20B9208AA0A920BE0E4
:109C70003AA2F9E75B46089AFEF766FB0B9B9B5CF2
:109C80000A9A521E0A92137050EA0102F2D10A98FF
:109C9000ADEB000000F1200B600702D524F4803406
:109CA00001E04FF00109D94502DDA9EB0B0000E00E
:109CB000002000EB0B0141440890AAEB010AE003ED
:109CC00006D4DDE90F232146504600F063F8064430
:109CD0004FF0000908E009A911F80900DDE90F12A9
:109CE000904709F10109761CC145F4DBE0030CD56E
:109CF000DDE90F232146504600F04CF8064404E00D
:109D0000DDE90F1230209047761C0899481E089014
:109D10000029F5DC08E00A980A990078491C0A91A4
:109D2000DDE90F129047761CBBF10001ABF1010B8E
:109D3000F1DC21465046DDE90F2300F019F8064416
:109D40006D1C1BE6092801003031323334353637BB
:109D50003839616263646566000000003031323377
:109D60003435363738394142434445460000000017
:109D70002DE9F041044600251E461746880404D408
:109D800005E039462020B0476D1C641EF9D52846F1
:109D9000BDE8F0812DE9F041044600251E469046BD
:109DA000C80301D5302700E02027880404D505E04A
:109DB00041463846B0476D1C641EF9D52846BDE8BB
:109DC000F0810146AEE000BF00BF00BF00BF00BF92
:109DD00000BF00BF00BF00BF00BF00BF00BF00BF8B
:109DE00000BF00BF00BF00BF00BF00BF00BF00BF7B
:109DF00000BF00BF00BF00BF00BF00BF00BF00BF6B
:109E000000BF00BF00BF00BF00BF00BF00BF00BF5A
:109E100000BF00BF00BF00BF00BF00BF00BF00BF4A
:109E200000BF00BF00BF00BF00BF00BF00BF00BF3A
:109E300000BF00BF00BF00BF00BF00BF00BF00BF2A
:109E400000BF00BF00BF00BF00BF00BF00BF00BF1A
:109E500000BF00BF00BF00BF00BF00BF00BF00BF0A
:109E600000BF00BF00BF00BF00BF00BF00BF00BFFA
:109E700000BF00BF00BF00BF00BF00BF00BF00BFEA
:109E800000BF00BF00BF00BF00BF00BF00BF00BFDA
:109E900000BF00BF00BF00BF00BF00BF00BF00BFCA
:109EA00000BF00BF00BF00BF00BF00BF00BF00BFBA
:109EB00000BF00BF00BF00BF00BF00BF00BF00BFAA
:109EC00000BF00BF00BF00BF00BF00BF00BF00BF9A
:109ED00000BF00BF00BF00BF00BF00BF00BF00BF8A
:109EE00000BF00BF00BF00BF00BF00BF00BF00BF7A
:109EF00000BF00BF00BF00BF00BF00BF00BF00BF6A
:109F000000BF00BF00BF00BF00BF00BF00BF00BF59
:109F100000BF00BF00BF00BF00BF00BF00BF00BF49
:109F20004A1E91B200293FF74EAF70470121012030
:109F30000B4A12680AB1002011E00A4A12680AB1FD
:109F400000200CE0084A12680AB1002007E0074A26
:109F50001368074A1268521E934200D102207047CC
:109F6000E085FF1F3C81FF1F3881FF1F0886FF1F10
:109F70002881FF1F1FB5002004E04106090E0DF8DF
:109F80000010401C1028F8D3FEF7EEFB03E04FF45E
:109F9000FA7001F00FFCFAE713B50C46FF2301221B
:109FA00069460248FFF72EFC00981CBD00D0014016
:109FB00000B587B001A8FEF7D1FD0220ADF806007C
:109FC0000020ADF8040001AA4FF480610220FEF7E2
:109FD00021FD01AA4FF400610220FEF71BFD4FF4A2
:109FE00080610220FEF7A0FD4FF400610220FEF721
:109FF0009BFD07B000BD70B506460024FFF7FAF9D7
:10A0000000251BE04FF400610220FEF76BFD0520E8
:10A01000FFF7D7FE4FF400610220FEF785FD6006D2
:10A02000040E4FF480610220FEF74EFD08B1601C63
:10A03000C4B20520FFF7C5FE681CC5B2082DE1DBE0
:10A04000204670BD70B50446FFF7E1F94FF400619A
:10A050000220FEF747FD002521E004F0800028B132
:10A060004FF480610220FEF75FFD04E04FF4806151
:10A070000220FEF737FD6006040E0520FFF7A1FE63
:10A080004FF400610220FEF74FFD0520FFF799FE17
:10A090004FF400610220FEF725FD681CC5B2082DB3
:10A0A000DBDB70BD10B5FFF7B2F94FF48061022021
:10A0B000FEF73AFD4FF400610220FEF735FD052062
:10A0C000FFF77FFE4FF480610220FEF70BFD0520B5
:10A0D000FFF777FE4FF400610220FEF703FD10BD8D
:10A0E00010B5FFF794F94FF400610220FEF7FAFC77
:10A0F0004FF480610220FEF7F5FC0520FFF761FEBA
:10A100004FF400610220FEF70FFD4FF48061022042
:10A11000FEF70AFD0520FFF754FE10BD10B5C82458
:10A12000FFF775F94FF480610220FEF7FDFC012076
:10A13000FFF747FE4FF400610220FEF7F5FC012017
:10A14000FFF73FFEFFF756F909E0601E84B21CB925
:10A15000FFF7C6FF012010BD0120FFF732FE4FF4CC
:10A1600080610220FEF7B0FC0028EED14FF40061C0
:10A170000220FEF7B7FC0020EDE700001CB5C72069
:10A18000FEF7B4FD01F074F800F0B4FF00F058F8E9
:10A1900000F086F8C720FEF7F1FD002002210346FB
:10A1A0000A02CDE9001017A11A4801F03BFF002078
:10A1B000022103460A02CDE9001017A1194801F057
:10A1C00031FF0020032103464FF40072CDE9001057
:10A1D00015A1184801F026FF01F07AFB11E000BF3D
:10A1E000BFF34F8F1448006800F4E0601349084340
:10A1F000001D11490860BFF34F8F00BF00BF00BFB3
:10A20000FDE7ECE76E6361393535355F7461736B7B
:10A2100000000000E1A300006563363030675F7422
:10A2200061736B00759F00006D70755F7461736B77
:10A230000000000071A200000CED00E00000FA0533
:10A2400000B587B001A8FEF789FC0220ADF8060032
:10A250000020ADF8040001AA04210520FEF7DAFB76
:10A2600001AA4FF440410220FEF7D4FB07B000BD25
:10A2700004210520FEF758FC4FF480410220FEF730
:10A2800053FC4FF47A7001F095FA4FF480410220AC
:10A29000FEF728FC03E04FF4FA7001F08BFAFAE7BE
:10A2A00010B5FFF785FE10BD2DE9F04107460C46BD
:10A2B00015461E464FF00008FFF7F4FE3846FFF73C
:10A2C000C1FEFFF72BFF80462846FFF7BBFEFFF7D6
:10A2D00025FF8046FFF7E6FE2046FFF7B3FEFFF7B7
:10A2E0001DFF80460020FFF786FE3070FFF7F8FE66
:10A2F0000020BDE8F081F8B504460E4615461F461D
:10A3000000200090012E01DC802D00DDF8BDD6B9C3
:10A3100044F001016B4602222046FFF7C5FF012FE2
:10A3200008D19DF8001041EA05022046022100F004
:10A3300072F824E09DF8001021EA0502204602216F
:10A3400000F069F81BE0012E19D144F001016B46C1
:10A3500003222046FFF7A8FF012F08D19DF8001027
:10A3600041EA05022046032100F055F807E09DF878
:10A37000001021EA05022046032100F04CF800BF3E
:10A38000C4E7F8B504460D46164600200090012D9E
:10A3900001DC802E00DDF8BD7DB944F001016B4683
:10A3A00006222046FFF780FF9DF8001021EA0602F2
:10A3B0002046062100F02FF810E0012D0ED144F0C8
:10A3C00001016B4607222046FFF76EFF9DF8001043
:10A3D00021EA06022046072100F01DF800BFDAE757
:10A3E0000F2200214020FFF7CCFF13E001230F22B2
:10A3F00000214020FFF77FFF4FF4FA7001F0DAF9F7
:10A4000000230F2219464020FFF775FF4FF4FA7022
:10A4100001F0D0F9EAE72DE9F04106460C46154671
:10A420000127FFF73FFE3046FFF70CFEFFF776FEF1
:10A4300007462046FFF706FEFFF770FE0746284650
:10A44000FFF700FEFFF76AFE0746FFF749FE002010
:10A45000BDE8F0812DE9F04105460E462648076823
:10A4600026480068001D00F061FF50B923480068CD
:10A4700090F82C1001208840214909688143204828
:10A480000160681CD8B9D6B11E4948681B490968E3
:10A4900088601A4982680968CA6018490968091DF4
:10A4A0008268516015490968091D8160154A134980
:10A4B00009684A6111460968491C11601AE07C1953
:10A4C0000E4800684460BC4207D20C480168091D70
:10A4D0000D48006800F04EFF0CE008480168091DB7
:10A4E0000A48006800F046FF09480068844201D22B
:10A4F00007480460BDE8F0812C81FF1F1881FF1F11
:10A500003081FF1F0886FF1F2081FF1F1C81FF1F56
:10A510004881FF1F10B5044600F046FF314800682F
:10A52000401C304908603048006840B92E4804603B
:10A530000846006801280DD100F054FA0AE02B48C3
:10A54000006838B928480068C06AE16A884201D8C2
:10A550002548046026480068401C254908600846D4
:10A560000068606494F82C10012088402149096833
:10A57000084320490860E16A01EB81011E4A02EBB1
:10A5800081014868A0608268E260211D8268516094
:10A590008160E16A01EB8101174A02EB810262618D
:10A5A000E16A01EB8101144A52F82110491CE26A68
:10A5B00002EB8202104B43F8221000F01FFF0B4801
:10A5C000006868B108480068C06AE16A884207D23A
:10A5D0004FF0805009490860BFF34F8FBFF36F8F72
:10A5E00010BD00002881FF1F1881FF1F3481FF1F4D
:10A5F0004481FF1F3081FF1F3883FF1F04ED00E0FF
:10A6000010B500F0D1FE10480068D0B90F4800F036
:10A61000A1FE0F4800F09EFE0C480E4908600C4851
:10A620000D49086000220C210A2001F0C1FA0649F8
:10A6300008600846006820B108A10348006801F0DE
:10A6400063F800F0DBFE10BD6081FF1F1C86FF1F5A
:10A650003086FF1F5881FF1F5C81FF1F546D7251B0
:10A660000000000010B516E000F09EFE0C48C06827
:10A67000C468201D00F05AFE0A480068401E0949BF
:10A68000086009480068401E0749086000F0B6FEEF
:10A69000204600F05FF8044800680028E4D110BDAF
:10A6A000F485FF1F2881FF1F2481FF1F70B504461A
:10A6B0000D46206C70B1216CE0680144E160D4E982
:10A6C0000210884201D32168E1602846226CE168CB
:10A6D000FDF77AFE70BD2DE9F04104460F461546A0
:10A6E0004FF00008A66B206C48B9206800282CD1D8
:10A6F000A06801F0BBFD80460020A06025E07DB988
:10A700003946226C6068FDF75FFE216C6068084482
:10A710006060D4E90101884217D32068606014E0CA
:10A720003946226CE068FDF74FFE216CE068411A63
:10A73000E1602168E068884203D2216CA068411A78
:10A74000E160022D01D106B1761E701CA063404667
:10A75000BDE8F08110B50446206B00F06DFE204688
:10A7600000F06AFE10BD0000002101220C4B1B68A6
:10A77000012B00D901210B4A1268D26A0AB10020CC
:10A780000DE0094A1268012A01D9002007E009B149
:10A79000002004E0054A1268054B1B68D01A704778
:10A7A0003081FF1F1881FF1F3883FF1F4881FF1F63
:10A7B0002C81FF1F0146084A126812680AB901225B
:10A7C00000E000220A600A6822B9034A1268D268CF
:10A7D000106800E0002070475881FF1F30B54FF42B
:10A7E000F043174800F007042CB1C01D20F007000B
:10A7F000134C041B1B1B0246124C22600024114DFB
:10A800006C60D018083820F007000F4C206000243E
:10A810000D4D2D686C600C4D2D682C601146441A4E
:10A820004C60094C24680C60084D4C682C60084D45
:10A830004C682C604FF00044064D2C6030BD000089
:10A840004486FF1F6C81FF1F7481FF1F7C81FF1FE7
:10A850007881FF1F8881FF1F00BFFFF703FF1948A2
:10A860000068012807D94FF0805017490860BFF3EE
:10A870004F8FBFF36F8FFFF777FF0446022C20D373
:10A8800001F094F81148006811490968884201D321
:10A89000012000E0002050B900BF502080F3118853
:10A8A000BFF34F8FBFF36F8F00BF00BFFEE7FFF70F
:10A8B0005BFF0446022C02D3204600F043FE01F069
:10A8C000DFFDCAE73883FF1F04ED00E04881FF1F6A
:10A8D0002C81FF1F2DE9F04106460D46174698468C
:10A8E000069C0DB9246000E02760E6632564012121
:10A8F000204601F091F984F850800020A064BDE862
:10A90000F0812DE9F05F82460F4690469B460A9EF5
:10A910000C9C4FEA8801A522206BFDF767FDA8F18A
:10A920000100216B01EB800929F0070909F00700FC
:10A9300008B9012000E0002050B900BF502080F38A
:10A940001188BFF34F8FBFF36F8F00BF00BFFEE7CB
:10A9500087B1002507E0795D04F134004155785D49
:10A9600000B902E06D1C102DF5D300BF002143207B
:10A97000015502E0002084F83400202E01D201208D
:10A9800000E0002050B900BF502080F31188BFF3D1
:10A990004F8FBFF36F8F00BF00BFFEE7202E00D3A5
:10A9A0001F26E662E66400202065201D00F0DFFC23
:10A9B00004F1180000F0DBFC2461C6F12000A06166
:10A9C00064620020606584F858005A465146484643
:10A9D00000F07AFB20600B9808B10B980460BDE88A
:10A9E000F09F000010B5002407E004EB84010F4A3B
:10A9F00002EB810000F0AEFC641C202CF5D30C4867
:10AA000000F0A8FC0B4800F0A5FC0B4800F0A2FCED
:10AA10000A4800F09FFC0A4800F09CFC04480949E1
:10AA2000086004480849086010BD00003883FF1F13
:10AA3000B885FF1FCC85FF1FE085FF1FF485FF1F32
:10AA40000886FF1F1C81FF1F2081FF1F10B50146D4
:10AA5000164800E0006803688B42FBD30246436857
:10AA600013448B4204D143684C682344436001463D
:10AA70000A464B6813440468A34211D10C4C036886
:10AA80002468A34208D04B680468646823444B6080
:10AA900003681B680B6005E0054B1B680B6001E059
:10AAA00003680B60884200D0016010BD6C81FF1FFD
:10AAB0007481FF1F2DE9F04104460D4616461F46DE
:10AAC0004FF0000865602461B5420CD8F01BA16905
:10AAD000884202D34FF0010811E0211D09480068A7
:10AAE00000F048FC0BE0BE4204D2BD4202D34FF05E
:10AAF000010804E0211D0448006800F03BFC4046CA
:10AB0000BDE8F0815C81FF1F5881FF1F70B50546CD
:10AB100000F04AFCA86B08B9012400E0002400F012
:10AB20006DFC204670BDF1B50098846C002654B9C8
:10AB300000BF502080F31188BFF34F8FBFF36F8F9A
:10AB400000BF00BFFEE7A06BE16B884201D201208D
:10AB500000E0002050B900BF502080F31188BFF3FF
:10AB60004F8FBFF36F8F00BF00BFFEE7A06BE16B9D
:10AB700088422CD294F94550002269462046FFF7BE
:10AB8000AAFD0646681C60B9606A08B9012000E0A9
:10AB90000020D8B904F1240001F0E0FBB0B1012697
:10ABA00014E07F2D01D0012000E0002050B900BF4B
:10ABB000502080F31188BFF34F8FBFF36F8F00BF1A
:10ABC00000BFFEE7681C40B284F8450000BF304675
:10ABD000F8BD000070B505460E460E480068C06816
:10ABE000C468201D00F0A2FB94F8280000F00400C7
:10ABF00028B132462946204600F0D6F805E094F800
:10AC0000280000F0FE0084F828002046216A8847CA
:10AC100070BD00005881FF1F7FB57FE001980028BC
:10AC20007CDB039C606908B9012000E0002010B9BA
:10AC3000201D00F07BFB684600F0E2F80546019815
:10AC40000A2869D2DFE800F06805072E36580608A2
:10AC50002F3700BF00BF00BF94F8280040F001006C
:10AC600084F828000298A269811803462A462046E3
:10AC7000FFF720FFA8B194F8280000F0040038B1D5
:10AC80000298A26981182A46204600F08DF805E056
:10AC900094F8280000F0FE0084F828002046216A7D
:10ACA00088473AE000BF94F8280000F0FE0084F8DE
:10ACB000280032E000BF94F8280040F0010084F83A
:10ACC00028000298A061A06908B1012000E00020DE
:10ACD00050B900BF502080F31188BFF34F8FBFF3EE
:10ACE0006F8F00BF00BFFEE7A06941192B462A46BF
:10ACF0002046FFF7DFFE10E094F8280000F0020085
:10AD000018B9204600F098FB05E094F8280000F000
:10AD1000FE0084F8280000E000BF00BF002201A967
:10AD20000348006801F082F800287FF477AF7FBD08
:10AD30006081FF1FF8B505460C4600F037FE6846F7
:10AD400000F05EF80646009820BB44B9B54206D82C
:10AD500001F096FB31462846FFF73CFF1CE03CB172
:10AD60000E480068006808B9012000E00020044691
:10AD7000A91B22460A48006800F0F6FC01F080FB9F
:10AD800050B94FF0805007490860BFF34F8FBFF3B1
:10AD90006F8F01E001F074FBF8BD00005C81FF1FC4
:10ADA0006081FF1F04ED00E070B504460D461646B5
:10ADB00004E0A06905442046216A8847A06941193A
:10ADC0002B4632462046FFF775FE0028F1D170BDB4
:10ADD00009480068006808B9012000E0002020B19F
:10ADE0004FF0FF300549086005E003480068C0687F
:10ADF00000680249086070471C81FF1F4881FF1FDF
:10AE000070B5044601F04EF90546074800688542D2
:10AE100004D200F00BF80120206001E00020206047
:10AE200001480560284670BD6881FF1F70B508E0C5
:10AE30000D480068C06804684FF0FF312046FFF7F6
:10AE4000C9FE09480068006808B9012000E0002038
:10AE50000028EDD0044805680448006802490860ED
:10AE60000248056070BD00005881FF1F5C81FF1F14
:10AE70000E480068401C08B9012000E0002050B9CD
:10AE800000BF502080F31188BFF34F8FBFF36F8F47
:10AE900000BF00BFFEE700BF502080F31188BFF362
:10AEA0004F8FBFF36F8F00BF00BFFEE78C81FF1F86
:10AEB00008B500BF6846FFF77DFC044620460099B0
:10AEC000FFF738FFFFF7A8FEF4E770B5044600F07F
:10AED0006BFA94F9455019E0A06C30B12046FFF7A9
:10AEE00022FE88B100F0A0FC0EE0606A08B90120E3
:10AEF00000E0002038B904F1240001F02FFA18B165
:10AF000000F092FC00E003E0681E45B2002DE3DC97
:10AF100000BFFF2084F8450000F070FA00F044FA0A
:10AF200094F9445010E0206908B9012000E00020A5
:10AF300048B904F1100001F011FA08B100F074FCF6
:10AF4000681E45B200E001E0002DECDC00BFFF20F0
:10AF500084F8440000F052FA70BD00002DE9F04181
:10AF600004464FF0000800F021FD5148006808B980
:10AF7000FFF734FC4F480068204000287ED13CB3E6
:10AF800004F10800A04223D9083404F0070000B3FC
:10AF900004F00700C0F108002044A04216D904F0D4
:10AFA0000700C0F10800044404F0070008B90120BC
:10AFB00000E0002068B900BF502080F31188BFF383
:10AFC0004F8FBFF36F8F00BF00BFFEE7002400E08C
:10AFD0000024002C54D038480068844250D8374EA2
:10AFE0003046056801E02E462D686868A04202D20E
:10AFF00028680028F7D12E480068854240D0306884
:10B0000000F10808286830606868001B102819D90A
:10B010002F1907F0070008B9012000E0002050B9FF
:10B0200000BF502080F31188BFF34F8FBFF36F8FA5
:10B0300000BF00BFFEE76868001B78606C603846A0
:10B04000FFF704FD1C4968680968081A1A49086076
:10B05000084600681A490968884203D21648006801
:10B060001749086013496868096808436860002048
:10B07000286014480068401C124900E000E00860A5
:10B0800001F0FEF908F0070008B9012000E00020F7
:10B0900050B900BF502080F31188BFF34F8FBFF32A
:10B0A0006F8F00BF00BFFEE74046BDE8F0810000A3
:10B0B0007481FF1F8881FF1F7881FF1F6C81FF1F34
:10B0C0007C81FF1F8081FF1F001F4FF08073036092
:10B0D000001F21F001030360001F054B03601438BB
:10B0E0000260001F6FF00203036020387047000009
:10B0F00071AE000000B595B02A2240210120FDF775
:10B10000FDFC2B2280210120FDF7F8FC28224FF4C2
:10B1100000710120FDF7F2FC29224FF4807101201B
:10B12000FDF7ECFC01218804FDF744FC0AA8FEF7BA
:10B13000BBF901200A9000200B900C900E900F900C
:10B140004CF2080010904FF4806011900020129093
:10B15000149040F27510ADF800000620ADF8020022
:10B160003C4801906846FDF70BFDBDF90200FEF773
:10B17000B3FBBDF902000E21FEF7CEFBBDF90200C4
:10B18000FEF7B8FB0AA93448FEF752F901214FF443
:10B190001030FDF7FFFB02A8FDF72AFB0120069007
:10B1A00000020790002005900120089000200990DF
:10B1B0002A4803902848049002AA00212848FDF755
:10B1C000A2FA08B100BFFEE740F24F112548FDF793
:10B1D0005EF94FF4805002900020089004200990FE
:10B1E0001D4803902048049002AA01211C48FDF745
:10B1F0008AFA08B100BFFEE74FF4A7711948001D95
:10B20000FDF745F92320ADF800000520ADF8020058
:10B21000164801906846FDF7B3FCBDF90200FEF741
:10B220005BFBBDF902000F21FEF776FBBDF90200C2
:10B23000FEF760FB01210A48FDF763FA01220021B5
:10B240000748FDF74AFA012211460548FDF745FA7D
:10B2500015B000BD2D940000000002401480FF1FB7
:10B260000030054014080140A881FF1F1588000028
:10B270000EB52C492C48FDF7A4F901220321052025
:10B28000FDF7A8FB02A8FDF71BFA00208DF80A00C5
:10B2900030208DF8090000208DF8080005208DF879
:10B2A0000B0002A8FDF7EAF96846FDF761F90020F6
:10B2B0008DF800000190019820F0030001906321B7
:10B2C000019861F310200190019820F0704000F186
:10B2D000E0400190019820F0706000F1E060019082
:10B2E000019820F4700000F5E0000190019820F032
:10B2F000800001906846FDF71BF9002211460320EB
:10B30000FEF7ECF8012211460420FEF7E7F80320CF
:10B31000FDF788FA4FF44050FDF712FC0520FDF7C9
:10B320005AF90EBD102211007777770701460A6996
:10B33000D1E901309860D1E9010358605068884232
:10B3400001D188685060002008611068401E1060BC
:10B350001068704700F1080141604FF0FF318160D3
:10B3600000F10801C1600161002101607047002106
:10B370000161704710B502460B685C1C0CB910697E
:10B3800007E002F1080000E04068446824689C423D
:10B39000FAD944684C604C68A160886041600A61D9
:10B3A0001468641C146010BD00BF502080F3118825
:10B3B000BFF34F8FBFF36F8F00BF0E480068401C74
:10B3C0000C49086008460068012812D10A48006844
:10B3D000C0B208B9012000E0002050B900BF5020E1
:10B3E00080F31188BFF34F8FBFF36F8F00BF00BF93
:10B3F000FEE770478C81FF1F04ED00E00D480068F8
:10B4000050B900BF502080F31188BFF34F8FBFF3B6
:10B410006F8F00BF00BFFEE706480068401E054969
:10B4200008600846006820B9002080F3118800BF3A
:10B4300000BF70478C81FF1F70B506463546002E51
:10B4400044D0083D2C46224960680968084008B18C
:10B45000012000E0002050B900BF502080F3118887
:10B46000BFF34F8FBFF36F8F00BF00BFFEE72068B1
:10B4700008B9012000E0002050B900BF502080F33F
:10B480001188BFF34F8FBFF36F8F00BF00BFFEE780
:10B490000F49606809680840C0B12068B0B90C491C
:10B4A000606809688843606000F080FA0949606854
:10B4B00009680844074908602046FFF7C7FA0648AC
:10B4C0000068401C0449086000F0DAFF70BD00000D
:10B4D0008881FF1F7881FF1F8481FF1F1548006846
:10B4E0004FF47A71B0FBF1F0134908600846006828
:10B4F0006FF07F41B1FBF0F0104908600D48006823
:10B50000B0FBF0F02D21B1FBF0F00D4908600020F8
:10B510004FF0E02108618861064800684FF47A71B5
:10B52000B0FBF1F0401E4FF0E021486107200861B8
:10B530007047000044FEFF1F9081FF1F9481FF1F92
:10B540009881FF1F2DE9F04104464E48006884426F
:10B5500001D94C4804684FF0E020006920F0010058
:10B560004FF0E021086108468169601E464A126872
:10B5700002FB001545480068854202D9434800682F
:10B580002D1A72B6BFF34F8FBFF36F8FFEF7CEFC4D
:10B5900080B94FF0E02080694FF0E0214861084613
:10B5A000006940F00100086137480068401E4861AA
:10B5B00062B665E04FF0E020456100204FF0E021E9
:10B5C00088610846006940F001000861A046B8F1B2
:10B5D000000F04D0BFF34F8F30BFBFF36F8F62B641
:10B5E000BFF34F8FBFF36F8F72B6BFF34F8FBFF3B1
:10B5F0006F8F06204FF0E02108610846006900F4D3
:10B600008030B8B120490968491E4FF0E0229269A4
:10B61000AA1A881A1D490968884203D31A49096879
:10B62000884202D918490968481E4FF0E021486154
:10B63000661E12E01448006860434FF0E0218969FB
:10B64000471A11480068B7FBF0F6701C0E490968EC
:10B650004843C01B4FF0E021486100204FF0E0213B
:10B6600088610846006940F001000861304600F03A
:10B670007DF905480068401E4FF0E021486162B640
:10B68000BDE8F0819481FF1F9081FF1F9881FF1F0B
:10B6900070B5FCF743FE0446102C16D304F1E020ED
:10B6A00090F8F05315480078854201DB012000E056
:10B6B000002050B900BF502080F31188BFF34F8F96
:10B6C000BFF36F8F00BF00BFFEE70D48006800F4B6
:10B6D000E0600C490968884201D8012000E00020A0
:10B6E00050B900BF502080F31188BFF34F8FBFF3D4
:10B6F0006F8F00BF00BFFEE770BD00009C81FF1F81
:10B700000CED00E0A081FF1F30B502460B4652B998
:10B7100000BF502484F31188BFF34F8FBFF36F8FA6
:10B7200000BF00BFFEE70021BBB1002012E00D4CBE
:10B7300004EBC0046468944203D10A4C04EBC001DA
:10B740000AE031B9074C54F8304014B9054C04EB09
:10B75000C001401C0A28EAD300BF09B10B604A604F
:10B7600030BD0000E882FF1F2DE9F04105460E467E
:10B7700017462C46FFF718FE94F94400401C10B9F8
:10B78000002084F8440094F94500401C10B90020C2
:10B7900084F84500FFF732FEA06B28B93A463146DF
:10B7A00004F1240000F062F82046FFF78EFBBDE8AC
:10B7B000F081000070B504460025D4B1124800683D
:10B7C00008B9012000E0002050B900BF502080F3EC
:10B7D0001188BFF34F8FBFF36F8F00BF00BFFEE72D
:10B7E00000F0E4F800212046FEF734FE00F048FEA9
:10B7F00005463DB94FF0805004490860BFF34F8FB4
:10B80000BFF36F8F70BD00005481FF1F04ED00E097
:10B8100003490968016003490968416070470000F5
:10B820004081FF1F2C81FF1F0120014908607047E4
:10B830003C81FF1F70B504460D4654B900BF50202F
:10B8400080F31188BFF34F8FBFF36F8F00BF00BF2E
:10B85000FEE70548016818312046FFF78BFD0121FE
:10B860002846FEF7F7FD70BD1881FF1F70B504462E
:10B870000E46154654B900BF502080F31188BFF31F
:10B880004F8FBFF36F8F00BF00BFFEE760680F49A7
:10B890000968C8610D49826809680A620B4909682C
:10B8A0001831826851600949096818318160074977
:10B8B00009688C622168491C21600DB14FF0FF3688
:10B8C00029463046FEF7C6FD70BD00001881FF1FF7
:10B8D0001CB51E4800210B468022CDE900101CA19A
:10B8E0001D4800F09FFB0446012C02D100F084FEAD
:10B8F0000446012C15D100BF502080F31188BFF3FE
:10B900004F8FBFF36F8F00BF4FF0FF3013490860B8
:10B9100001201349086000201249086000F094F8E3
:10B9200010E0601C08B1012000E0002050B900BF09
:10B93000502080F31188BFF34F8FBFF36F8F00BF8C
:10B9400000BFFEE7084800681CBD00004C81FF1FD7
:10B9500049444C450000000059A800004881FF1FE1
:10B960003481FF1F2C81FF1F5081FF1F0D49096883
:10B9700001440D4A1268914201D8012100E00021E2
:10B9800051B900BF502181F31188BFF34F8FBFF32E
:10B990006F8F00BF00BFFEE7024909680144014AFA
:10B9A000116070472C81FF1F4881FF1F024800680B
:10B9B000401C0149086070475481FF1F1D48006802
:10B9C00018B101201C49086032E000201A490860C3
:10B9D0001A480068B0FA80F0C0F11F0101EB810045
:10B9E000174A52F8200008B1012000E0002050B9A9
:10B9F00000BF502080F31188BFF34F8FBFF36F8FCC
:10BA000000BF00BFFEE701EB81020D4B03EB82009C
:10BA100042685268426000F108024368934202D1D2
:10BA20004268526842604268D268064B1A6000BFA2
:10BA3000704700005481FF1F3C81FF1F3081FF1FB2
:10BA40003883FF1F1881FF1F1CB5524800685249F8
:10BA5000884201D0012000E0002050B900BF5020F2
:10BA600080F31188BFF34F8FBFF36F8F00BF00BF0C
:10BA7000FEE7484800684849491E884201D0012035
:10BA800000E0002050B900BF502080F31188BFF3C0
:10BA90004F8FBFF36F8F00BF00BFFEE73F490846DF
:10BAA00000780190FF200A46107008460078009048
:10BAB0009DF8000000F0F0009DF80020904201D1B8
:10BAC000012000E0002050B900BF502080F3118811
:10BAD000BFF34F8FBFF36F8F00BF00BFFEE79DF82E
:10BAE000000000F050002E4A107007202D4A106010
:10BAF00009E02C480068401E2A4A10609DF80000AA
:10BB00004006000E00909DF8000000F080008028A4
:10BB1000EFD024480068C0F10700042801D10120BB
:10BB200000E0002050B900BF502080F31188BFF31F
:10BB30004F8FBFF36F8F00BF00BFFEE7194800684B
:10BB40000002184A10601046008800F4E06010609F
:10BB5000124A019810700F482030006840F47000BD
:10BB60000C49203108600846006840F070400860C9
:10BB7000FFF7B4FC00200C490860FCF797FB0B486A
:10BB8000006840F0404009490860FCF77BFB00205A
:10BB90001CBD000000ED00E071C20F4100E400E0B8
:10BBA0009C81FF1FA081FF1F8C81FF1F34EF00E0ED
:10BBB0002DE9F84305460E4617460024E5B1601E00
:10BBC000B0FBF5F0B04217D305FB06F010F1550FAE
:10BBD00012D805FB06F808F15400FFF7BFF9044638
:10BBE000B4B1A14609F154093B464A4631462846BC
:10BBF0000094FEF76FFE0BE054B900BF502080F3B5
:10BC00001188BFF34F8FBFF36F8F00BF00BFFEE7F8
:10BC10002046BDE8F88300002DE9F04105460E46B8
:10BC200001272C4654B900BF502080F31188BFF380
:10BC30004F8FBFF36F8F00BF00BFFEE7002C42D0D5
:10BC4000E06B00283FD04FF0FF31E06BB1FBF0F02C
:10BC5000216C884237D3FFF7A7FBD4E90F12206885
:10BC600001FB0200A0600020A06320686060E06B20
:10BC7000401E226C216800FB0211E160FF2084F865
:10BC8000440084F845009EB9206908B9012000E00D
:10BC90000020A8B904F1100000F060FB80B14FF063
:10BCA000805013490860BFF34F8FBFF36F8F07E0D9
:10BCB00004F11000FFF74EFB04F12400FFF74AFBEC
:10BCC000FFF79CFB00E000270FB1012000E00020FF
:10BCD00050B900BF502080F31188BFF34F8FBFF3DE
:10BCE0006F8F00BF00BFFEE73846BDE8F08100005F
:10BCF00004ED00E02DE9F84F80468B4615461E46C0
:10BD0000444654B900BF502080F31188BFF34F8FD1
:10BD1000BFF36F8F00BF00BFFEE7BBF1000F01D183
:10BD2000206C08B9012000E0002050B900BF50206D
:10BD300080F31188BFF34F8FBFF36F8F00BF00BF39
:10BD4000FEE7022E02D1E06B012801D1012000E0C4
:10BD5000002050B900BF502080F31188BFF34F8FEF
:10BD6000BFF36F8F00BF00BFFEE7FFF791FC00BF7E
:10BD70005021EFF3118081F31188BFF34F8FBFF390
:10BD80006F8F00BF0746A06BE16B884201D3022E84
:10BD900042D194F945A0A06B009032465946204606
:10BDA000FEF799FC0AF10100E0B9A06C58B1022E2F
:10BDB00001D1009868BB2046FEF7B5FE48B345B3F5
:10BDC0000120286025E0606A08B9012000E0002019
:10BDD000F8B904F1240000F0C1FAD0B1CDB10120CE
:10BDE000286016E0BAF17F0F01D0012000E00020AA
:10BDF00050B900BF502080F31188BFF34F8FBFF3BD
:10BE00006F8F00BF00BFFEE70AF1010040B284F867
:10BE100045004FF0010901E04FF0000900BF87F332
:10BE2000118800BF4846BDE8F88F00002DE9F741B2
:10BE300083B005460E464FF000082C4654B900BFAB
:10BE4000502080F31188BFF34F8FBFF36F8F00BF77
:10BE500000BFFEE70EB9206C08B9012000E0002009
:10BE600050B900BF502080F31188BFF34F8FBFF34C
:10BE70006F8F00BF00BFFEE700F004F908B9059816
:10BE800008B9012000E0002050B900BF502080F325
:10BE90001188BFF34F8FBFF36F8F00BF00BFFEE766
:10BEA00000BFFFF781FAA76BF7B131462046FEF7D6
:10BEB000FDFB781EA063206908B9012000E0002086
:10BEC00060B904F1100000F049FA38B14FF0805029
:10BED0002F490860BFF34F8FBFF36F8FFFF78EFAC4
:10BEE000012006B0BDE8F081059818B9FFF786FA81
:10BEF0000020F6E7B8F1000F04D101A8FFF788FC95
:10BF00004FF00108FFF77AFAFFF750FDFFF74CFA00
:10BF100094F94400401C10B9002084F8440094F9BE
:10BF20004500401C10B9002084F84500FFF766FA70
:10BF300005A901A800F02EF8F0B92046FEF7E6FDAD
:10BF4000A0B104F124000599FFF774FC2046FEF728
:10BF5000BCFF00F095FA0028A3D14FF080500C49A7
:10BF60000860BFF34F8FBFF36F8F9AE72046FEF74D
:10BF7000ACFF00F085FA94E72046FEF7A6FF00F03C
:10BF80007FFA2046FEF7C2FD00288AD00020A8E7ED
:10BF900004ED00E070B505460C4655B900BF5020D1
:10BFA00080F31188BFF34F8FBFF36F8F00BF00BFC7
:10BFB000FEE754B900BF502080F31188BFF34F8FC4
:10BFC000BFF36F8F00BF00BFFEE7FFF7EDF9134827
:10BFD00002686868131A2068401C08B9002619E036
:10BFE0000F4928680968884206D06868904203D8DB
:10BFF0000126002020600DE02068984207D92068C3
:10C00000C01A20602846FFF703FC002602E000204B
:10C0100020600126FFF7F2F9304670BD2C81FF1F2A
:10C020004081FF1F2DE9FF4F85B0804689461746A6
:10C03000DDE912ABB800FEF791FF064656B15C2071
:10C04000FEF78CFF04460CB1266304E03046FFF790
:10C05000F3F900E000247CB10020CDE900ABCDE98C
:10C0600002403A4649464046089BFEF74AFC2046B5
:10C07000FEF750FA012501E04FF0FF35284609B0E0
:10C08000BDE8F08F0549096809B9012005E00449B8
:10C09000096809B9022000E0002070473481FF1FC1
:10C0A0005481FF1F01490868704700002C81FF1F61
:10C0B0002DE9F0414FF000086148006800287DD16B
:10C0C00060480068451C5F48056015BB5E48006815
:10C0D000006808B9012000E0002050B900BF5020DE
:10C0E00080F31188BFF34F8FBFF36F8F00BF00BF86
:10C0F000FEE75548076855480068534908605348AB
:10C10000076053480068401C51490860FEF760FE14
:10C1100000BF50480068854277D300BF4A48006896
:10C12000006808B9012000E0002020B14FF0FF3086
:10C130004849086068E044480068C068C4686668A8
:10C14000B54202D2434806605EE06069D4E902125B
:10C150008A60D4E902214A60211D42688A4201D1E5
:10C16000E1684160002262610168491E0160A06AC5
:10C1700098B1A06AD4E907128A60D4E907214A601D
:10C1800004F1180142688A4201D1216A416000220B
:10C19000A2620168491E016000BF94F82C100120C2
:10C1A00088402D49096808432B490860E16A01EB82
:10C1B00081012A4A02EB8101486800E037E0A06073
:10C1C0008268E260211D826851608160E16A01EB52
:10C1D0008101224A02EB81026261E16A01EB810185
:10C1E0001E4A52F82110491CE26A02EB82021B4BE4
:10C1F00043F822101A49E06A0968C96A88428DD357
:10C200004FF001088AE700E000BF15480068C06AE7
:10C2100000EB8000114951F82000012801D94FF0AE
:10C2200001081048006808B14FF0010804E00E480A
:10C230000068401C0C4908604046BDE8F0810000E1
:10C240005481FF1F2C81FF1F1C81FF1F2081FF1FB6
:10C250004081FF1F4881FF1F3081FF1F3883FF1F70
:10C260001881FF1F3C81FF1F3881FF1F70B50546F5
:10C270002C460026002D68D035480068844201D144
:10C28000012000E0002050B900BF502080F3118849
:10C29000BFF34F8FBFF36F8F00BF00BFFEE7206D6E
:10C2A00050B900BF502080F31188BFF34F8FBFF308
:10C2B0006F8F00BF00BFFEE7206D401E2065E16C60
:10C2C000E06A884241D0206D00283ED1201DFFF752
:10C2D0002DF840B994F82C10012088401D490968B8
:10C2E00081431C480160E06CE062E06AC0F120001C
:10C2F000A06194F82C100120884016490968084371
:10C3000014490860E16A01EB8101134A02EB8101E3
:10C310004868A0608268E260211D82685160816087
:10C32000E16A01EB81010C4A02EB81026261E16A80
:10C3300001EB8101084A52F82110491CE26A02EB24
:10C340008202054B43F822100126304670BD0000E2
:10C350001881FF1F3081FF1F3883FF1F70B506460D
:10C36000F068C46854B900BF502080F31188BFF34F
:10C370004F8FBFF36F8F00BF00BFFEE7A06AD4E905
:10C3800007128A60D4E907214A6004F11801426863
:10C390008A4201D1216A41600022A2620168491EDD
:10C3A00001603148006800283FD16069D4E9021279
:10C3B0008A60D4E902214A60211D42688A4201D183
:10C3C000E1684160002262610168491E016094F8E1
:10C3D0002C1001208840254909680843234908603A
:10C3E000E16A01EB8101224A02EB81014868A06009
:10C3F0008268E260211D826851608160E16A01EB20
:10C4000081011B4A02EB81026261E16A01EB810159
:10C41000174A52F82110491CE26A02EB8202144BBF
:10C4200043F82210FEF7D4FC10E012494868E0619E
:10C430008268226204F118018268516081600D4AAD
:10C44000A26211460968491C116000BF0A49E06AEE
:10C450000968C96A884204D9012501200749086092
:10C4600000E00025284670BD5481FF1F3081FF1F6A
:10C470003883FF1FE085FF1F1881FF1F3C81FF1FCE
:10C4800070B5002400265348006850B900BF502002
:10C4900080F31188BFF34F8FBFF36F8F00BF00BFD2
:10C4A000FEE7FEF781FF4B480068401E49490860DF
:10C4B0000846006800287DD147480068002879D0E8
:10C4C0005BE04648C068C468A06AD4E907128A6085
:10C4D000D4E907214A6004F1180142688A4201D177
:10C4E000216A41600022A2620168491E0160606900
:10C4F000D4E902128A60D4E902214A60211D42680F
:10C500008A4201D1E1684160002262610168491EEE
:10C51000016094F82C1001208840314909680843D3
:10C520002F490860E16A01EB81012E4A02EB81018B
:10C530004868A0608268E260211D82685160816065
:10C54000E16A01EB8101274A02EB81026261E16A43
:10C5500001EB8101234A52F82110491CE26A02EBE7
:10C560008202204B43F822101F49E06A0968C96A19
:10C57000884202D301201D4908601848006808B9A4
:10C58000012000E0002000289BD00CB1FEF720FC29
:10C590001748056865B100BFFFF78AFD10B101209B
:10C5A000124908606D1E002DF6D100201049086068
:10C5B0000E4800E009E0006838B1012630070D4957
:10C5C0000860BFF34F8FBFF36F8FFEF717FF304642
:10C5D00070BD00005481FF1F2881FF1FE085FF1FF1
:10C5E0003081FF1F3883FF1F1881FF1F3C81FF1F11
:10C5F0003881FF1F04ED00E01CB50024FEF700F8B1
:10C600000D48006850B10D4802210023CA01CDE950
:10C6100000100BA10C48FFF705FD044654B900BFFC
:10C62000502080F31188BFF34F8FBFF36F8F00BF8F
:10C6300000BFFEE720461CBD6081FF1F6481FF1F15
:10C64000546D722053766300B1AE00000001020306
:10C6500004050607080C1014182030401014181C8C
:10C660002028384884C600000080FF1FA801000071
:10C6700054840000D0C60000A881FF1FA8880000D5
:10C68000509900000115003CFF535049204D617343
:10C690007465722F536C617665206578616D706C7E
:10C6A000653A20436F6D6D756E69636174696F6E75
:10C6B000206265747765656E2074776F20626F61A4
:10C6C0007264732141023C1F0519AAAAAAAA00009C
:040000050000825124
:00000001FF
